:1000000008308A007E2D0000FF00030E8301A1004E
:100010007F08A0000A08A8008A01A00E0408A20018
:100020007708A3007808A4007908A5007A08A6003C
:100030007B08A700831383128B1E20280B193328FB
:10004000220884002308F7002408F8002508F90096
:100050002608FA002708FB0028088A00210E8300E2
:10006000FF0E7F0E09008A113528861A3B28290FBA
:100070003A283B28A90A86194128A90803194128CA
:10008000A9030B118A112028FF308316DD000F30E1
:10009000DE0083121308FF309300831614185228D1
:1000A00083124D285C0883121302031961288316FA
:1000B0005D080319DE03DD0B4928DE08031D49280E
:1000C00083128316DD08031D6C28DE08031D6C28CF
:1000D0000130F8006F286F280030F8006F28831275
:1000E00000349412FC127C086700FC117C08670045
:1000F0003130940040308316940014178312141288
:1001000005148316B5013508093C031C9228831297
:100110001308FF30930083161418902883128B283D
:10012000B50A832883120510130840309300831604
:1001300014189C28831297280430B400B4080319BB
:10014000AB2883121308930183161418A92883126D
:10015000A428B4039E2883121308953093008316B5
:100160001418B4288312AF280130DC008312442015
:10017000780BBD280130F8003E298316B501350FF4
:10018000C228EC28DC0183124420780BC828CA2836
:100190008316EC2813084130930083161418D228D4
:1001A0008312CD280430B400B4080319E128831267
:1001B0001308930183161418DF288312DA28B40376
:1001C000D42883121308FF30930083161418EA28EA
:1001D0008312E528B50ABF283508FD3C0318F52829
:1001E0000130F80083123E29831683120514130888
:1001F000FF30930083161418FF288312FA28831205
:10020000051013085030930083161418092983121F
:1002100004298312130893018316141811298312D9
:100220000C298312130893018316141819298312B9
:1002300014298312130802309300831614182229FC
:1002400083121D29831213089301831614182A2977
:100250008312252983121308FF3093008316141884
:10026000332983122E29DC0183124420780B3B2989
:100270000130F8003E2905140030F8008A159F2D42
:10028000031083165A08DB005908DA005808D90011
:10029000D801D90DDA0DDB0D83120510130851308A
:1002A000930083161418562983125129DB308400D9
:1002B0000008DC008312130883165C088312930085
:1002C00083161418652983126029DA308400000827
:1002D000DC008312130883165C08831293008316D4
:1002E0001418742983126F29D93084000008DC00A7
:1002F0008312130883165C08831293008316141864
:10030000832983127E2983121308930183161418FC
:100310008B298312862983121308FF3093008316DA
:100320001418942983128F29DC0183124420780B3E
:100330009C290130F800A829FE308316DC008312C6
:100340004420780BA6290130F800A8290030F800D5
:1003500000348316D8080319C32983121308FF3009
:10036000930083161418B6298312B1298312130837
:10037000FF30930083161418BF298312BA29D803BB
:100380008312A9298316831200341308FF309300C7
:1003900083161418CD298312C82983121308AA00C2
:1003A0001308FF30930083161418D8298312D32919
:1003B00083121308AB00003413084C3093008316EB
:1003C0001418E4298312DF2983121308930183167A
:1003D0001418EC298312E72983121308930183165A
:1003E0001418F4298312EF2983121308930183163A
:1003F0001418FC298312F72983121308930183161A
:100400001418042A8312FF2983121308FF30930063
:10041000831614180D2A8312082A83121308FF303A
:10042000930083161418162A8312112A83120514B6
:100430001308FF30930083161418202A83121B2AF6
:1004400083120034F701F801F901FA018316D00193
:10045000D101D201D3014F084E044D044C040319BD
:10046000612A2030D4000310C80DC90DCA0DCB0D70
:10047000D00DD10DD20DD30D4F085302031D4A2AC2
:100480004E085202031D4A2A4D085102031D4A2AF2
:100490004C085002031C5B2A4C08D0024D08031C78
:1004A0004D0FD1024E08031C4E0FD2024F08031C01
:1004B0004F0FD3020314F70DF80DF90DFA0DD40BFD
:1004C000332A0000D0308400831200342030831699
:1004D000E600E201E301E401E5015D08FA005C08E1
:1004E000F9005B08F8005A08F7000310771C862A09
:1004F0005E08E2075F0803185F0FE3076008031850
:10050000600FE40761080318610FE507E50CE40CD0
:10051000E30CE20CFA0CF90CF80CF70CE60B752A5C
:1005200083120034AE01AD018316DB01DA01D9017B
:10053000D80183124021E3308316D8008312A92109
:10054000C5218316B90183122B088316B8008312C4
:10055000AE00AD012A08AD070318AE0ADC218316F0
:10056000BB01BA0183122E088316B90083122D082D
:100570008316B8003B08DB003A08DA003908D900D6
:100580003808D8008312402105308316D800831222
:10059000A921C521B6012B08B500C5218316B901D3
:1005A00083122A088316B800FA0000308312B507B8
:1005B0000318B60A7A08B6072B08AC00C5218316C3
:1005C000B90183122B088316B800BB00BA0183124D
:1005D0002A0883163A078312B30083163B08831256
:1005E000B4000318B40AC5212A08F300E601E501A6
:1005F000E4012B08E300C5218316B90183122A0800
:100600008316B800FA0000308312E3077A08031853
:100610007A0FE407003003180130E50700300318B3
:100620000130E607C521C5218316B90183122B08C5
:100630008316B800FA00003083122A07E7007A0810
:10064000E800003003180130E807E901EA0106304C
:100650008316D8008312A921C521EE01ED01EC011A
:10066000EB018316BB01BA01B90183122B08831673
:10067000B8003A08FA003908F9003808F800F7011C
:10068000770883122A07EB007808EC000030031883
:100690000130EC077908ED00003003180130ED0758
:1006A0007A08EE00003003180130EE076E0883165A
:1006B000B70083126D088316B60083126C08831688
:1006C000B50083126B088316B4008312C52183160C
:1006D000BB01BA01B90183122B088316B8003A088E
:1006E000FA003908F9003808F800F7017708831292
:1006F0002A07EB007808EC00003003180130EC0703
:100700007908ED00003003180130ED077A08EE009B
:10071000003003180130EE076C08EE006B08ED00A6
:10072000EB01EC01831634088312EB0783163508BE
:100730000318350F9C2B9F2B8312EC07831636086A
:100740000318360FA42BA72B8312ED078316370847
:100750000318370FAC2BAF2B8312EE0783168312CF
:10076000C521C521C5218316BB01BA01B901831278
:100770002B088316B8003A08FA003908F90038083F
:10078000F800F701770883122A07EF007808F000D5
:10079000003003180130F0077908F1000030031829
:1007A0000130F1077A08F200003003180130F20737
:1007B00072088316B7007108B6007008B50083127E
:1007C0006F088316B4008312C521DC218316BB0198
:1007D000BA01B90183122B088316B8003A08FA004F
:1007E0003908F9003808F800F701770883122A075A
:1007F000EF007808F000003003180130F0077908A6
:10080000F100003003180130F1077A08F2000030DF
:1008100003180130F2077008F2006F08F100EF01D1
:10082000F001831634088312EF0783163508031886
:10083000350FF00736080318360FF107370803188D
:10084000370FF20772088312DA007108D9007008B6
:10085000D8006F08D70033082D07C7002E08C8003E
:1008600034080318340FC807C901CA01630D831681
:10087000B8008312640D8316B9008312650D8316C8
:10088000BA008312660D8316BB00B80DB90DBA0D00
:10089000BB0DB80DB90DBA0DBB0DB80DB90DBA0D24
:1008A000BB0DB80DB90DBA0DBB0DE030B805013068
:1008B00083123502F7003608FA000030031C0130BD
:1008C000FA02770883163807BC003908BD007A0899
:1008D00003187A0FBD073A08BE0000300318013034
:1008E000BE073B08BF00003003180130BF073F08B8
:1008F000CB003E08CA003D08C9003C08C800CF0133
:10090000CE01831236088316CD0083123508831674
:10091000CC00831222227808B0007708AF00E708E5
:10092000031D9B2CE808031D9B2CE908031D9B2C31
:10093000EA080319DC2C1030F4008316DD01DC0119
:10094000DB017308DA0083126A088316E100831260
:1009500069088316E000831268088316DF0083129B
:1009600067088316DE008312662277083307831632
:10097000B800831234088316B90078080318780F7A
:10098000B9077908BA00003003180130BA077A08AD
:10099000BB00003003180130BB0783122F088316F9
:1009A00038078312B100831639088312B200031886
:1009B000B20A3008B2071C2D2030F4008316DD0186
:1009C000DC01DB017308DA0083126E088316E10094
:1009D00083126D088316E00083126C088316DF0013
:1009E00083126B088316DE008312662277083307B2
:1009F0008316B800831234088316B90078080318E8
:100A0000780FB9077908BA00003003180130BA0727
:100A10007A08BB00003003180130BB0783122F088F
:100A2000831638078312B100831639088312B20087
:100A30000318B20A3008B2078316BB01BA01B90124
:100A40007308B8003B08DD003A08DC003908DB0019
:100A50003808DA0083126A088316E10083126908F5
:100A60008316E000831268088316DF00831267088C
:100A70008316DE008312662277083307B700340836
:100A8000B80078080318780FB8077908B900003063
:100A900003180130B9077A08BA0000300318013092
:100AA000BA078316BB01BA0183122E088316B90058
:100AB00083122D088316B8008312F901FA01310858
:100AC000831638078312CB00831639088312CC00B3
:100AD00032080318320FCC0783163A088312CD0070
:100AE00079080318790FCD0783163B088312CE00CF
:100AF0007A0803187A0FCE078A15A92DC83084000A
:100B000000080319902D0230F800F701F70B862D2D
:100B1000F80B852D9730F700F70B8C2D800B832D6C
:100B200000348316D0010730D1008312061203303F
:100B3000F700F70B992D83164F08F7005108F800BE
:100B40000319A62D0310F70CF80BA22D7718AC2D66
:100B500083128610AE2D831683128614061600307B
:100B6000051B0130013C031DC32D0130F700831626
:100B70005108F8000319C02D0310F70DF80BBC2D18
:100B80007708D0048312061283165108D103003A65
:100B90000319CC2D83129B2D5008F80083120034CA
:100BA00005148515941283168610831285108316FA
:100BB0004808CF008312912583164908CF0083127D
:100BC0009125CD308316CE004A08CF00831291259F
:100BD00083164E08840078088000CC30CE004B0885
:100BE000CF008312912583164E0884007808800078
:100BF00083128514831686148312941683164C0868
:100C0000F8004D08F9008312003405148514851589
:100C100002308316B400FA30C80083127E25831692
:100C2000B40B0B2E831205112130F700F70B162E93
:100C30000515A630F700F70B1B2E000002308316B7
:100C4000C800C901CA010430CB008312D02564302A
:100C50008316C80083127E25051A302E8316122EA5
:100C600001308316C80083127E2502308316C80027
:100C7000C9010830CA00CB018312D0250130831688
:100C8000C80083127E2502308316C8000B30C900CD
:100C9000831229088316CA00831229088316CB0001
:100CA0008312D02501308316C80083127E258A1551
:100CB000AC2D8316D201D1010310CD0DCE0DCF0D79
:100CC000D00DCD3084000008D7004E08CD004F086D
:100CD000CE005008CF00D001831247088316CD07FD
:100CE000831248080318480F762E792E8316CE07F4
:100CF000831249080318490F7E2E812E8316CF07D1
:100D000083124A0803184A0F862E892E8316D007AD
:100D1000831283165008DB004F08DA004E08D90012
:100D20004D08D8008312402183165708D80083123B
:100D3000A921C5218316D90183122B088316D80057
:100D4000DB00DA01FA0183122A0883165A07D10060
:100D50005B08D2000318D20A7A08D2078312C52191
:100D60008316D601D501D401D301D90183122B08F2
:100D70008316D800DB00DA01FA0183122A088316F1
:100D80005A07D3005B08D4007A0803187A0FD407F7
:100D9000D501D6015408D6005308D500D301D4019B
:100DA000F901FA015108D30752080318520FD4076A
:100DB00079080318790FD5077A0803187A0FD60730
:100DC0008312DC2183165308F7005408F8005508F5
:100DD000F9005608FA00831200347208DA0071082C
:100DE000D9007008D8006F08D7008316B701B60184
:100DF000B501B40183125A08DE005908DD00580815
:100E0000DC005708DB005E088316D00083125D0803
:100E10008316CF0083125C088316CE0083125B0812
:100E20008316CD00831259267A08DA007908D90092
:100E30007808D8007708D70057088316B8008312BF
:100E400058088316B900831259088316BA00831212
:100E50005A080F398316BB000130B4070318B50ACE
:100E60000319B60A0319B70A3B080F3C031C4A2FA3
:100E7000031DFA2E3A08FF3C031C4A2F031DFA2ECD
:100E80003908FF3C031C4A2F031DFA2E3808EE3C9C
:100E90000318FA2E3708DD003608DC003508DB00C1
:100EA0003408DA00E101E001DF0183122C08831627
:100EB000DE00831266227A08E2007908E1007808F1
:100EC000E0007708DF00DF0DE00DE10DE20DDF0D42
:100ED000E00DE10DE20DDF0DE00DE10DE20DDF0DA6
:100EE000E00DE10DE20DF030DF05FF30DF07031C00
:100EF000E007031CE107031CE2078A15B42DFF304D
:100F00008316B700B6008312E208031DE12FE10843
:100F1000031DE12F6008831637020318912F8312F7
:100F2000E12F031D992F360883125F020318E12F6A
:100F30008316BA01F61F9E2F0130BA00F61EA22FAB
:100F40000130BA06761EA62F0130BA06761DAA2FEA
:100F50000130BA060310F60D3A08F6047608F800D8
:100F60007808B800B80E0F30B805A03038078400F4
:100F7000000FBB2FDF2FA030380784000008800A45
:100F8000B9007508B907831203178E01831603137E
:100F90003908831203178D0083168C130C148312E7
:100FA0000C0883160313B701B600BB013808B5005F
:100FB000B4013408B6070318B70A3508B707832FFA
:100FC000831283163608F7003708F800F901FA0192
:060FD00083128A15DE2DDC
:10100000F801F901F701FA0183165008031D0B28B6
:101010004F08031925281030D1000310CD0DCE0D37
:10102000F70DFA0D50087A02031D18284F087702B1
:10103000031C21284F08F702031CFA035008FA0288
:101040000314F80DF90DD10B0D28000083128A1539
:1010500077281030F700FA018316D101CE0CCD0CA1
:10106000031C38284F08FA070318D10A5008D10783
:10107000D10CFA0CF90CF80CF70B2E2883128A15F8
:1010800087288316C601C501C401C30172088312F3
:10109000DA007108D9007008D8006F08D7008316ED
:1010A000370CFA00360CF900350CF800340CF70058
:1010B000FA0CF90CF80CF70CFA0CF90CF80CF70C0C
:1010C000FA0CF90CF80CF70C7708C9007808CA007C
:1010D0004A08CC004908CB004A08CE004908CD0098
:1010E000D00183122C088316CF00831200287908C0
:1010F0008316CA007808C9004A08CE004908CD0006
:10110000D00183122C088316CF0083122928790876
:101110008316C8007808C70047084B02C700480874
:10112000031C480F95284C0896284C02C800C90893
:10113000031D9D28CA080319D62883125A08DE0009
:101140005908DD005808DC005708DB005E088316EC
:10115000D00083125D088316CF0083125C088316CB
:10116000CE0083125B088316CD008A1183125926A4
:101170008A157A08DA007908D9007808D800770843
:10118000D70057088316C300831258088316C4007B
:10119000831259088316C50083125A080F39831623
:1011A000C60049080319CA03C903972846080E3C1C
:1011B0000318F228FF3A031DEF284508FE3C0318E8
:1011C000F228FF3A031DEF284408FE3C0318F228DA
:1011D000FF3A031DEF284308EF3C0318F2280230C2
:1011E000F800162B0230831257028316BF008312B9
:1011F00058088316C0000030031C0130C00283125F
:1012000059088316C1000030031C0130C10283124B
:101210005A088316C2000030031C0130C202831238
:101220002C08F700F801F901FA017A088316D000BA
:101230007908CF007808CE007708CD004208DD009D
:101240004108DC004008DB003F08DA005008E100FC
:101250004F08E0004E08DF004D08DE008A118312BF
:1012600066228A157A088316C2007908C1007808B8
:10127000C0007708BF0083124B088316BF07831294
:101280004C0803184C0F452948298316C0078312C0
:101290004D0803184D0F4D2950298316C10783129D
:1012A0004E0803184E0F552958298316C20783127A
:1012B0008316F901FA014708BF0748080318480FC9
:1012C000C00779080318790FC1077A0803187A0F45
:1012D000C2074208DB004108DA004008D9003F0895
:1012E000D8008A11831240218A15831634080F39D9
:1012F000CD0035080039CE0036080039CF00370858
:101300000039D0004D0DD1004E0DD2004F0DD3004D
:10131000500DD400D10DD20DD30DD40DD10DD20D61
:10132000D30DD40DD10DD20DD30DD40DF030D10588
:101330005108D8008A118312A9218A158A11C52162
:101340008A15AA08031DAC298A11DC218A150030F0
:10135000F8008316162B83122A08E53C0319102B7C
:1013600003308316D8008A118312A9218A158A11A5
:10137000C5218A152A088316B80083122B08831604
:10138000B9008A118312C5218A152A088316BA006A
:1013900038086D3C0319D82938084D3C0319D82961
:1013A0003808573C0319D8293808773C031DEC2925
:1013B0003908503C0319E8293908703C0319E82919
:1013C0003908413C0319E8293908613C031DEC291F
:1013D0003A08333C0319F4293A08563C0319F42916
:1013E0003A08763C031D0F2B0430D8008A11831273
:1013F000A9218A158A11C5218A157408203C031D6C
:101400001D2A8316CE0183122B088316CD00D0002F
:10141000CF0183122A0883164F07BB005008BC0077
:10142000003003180130BC07BD01BE013C08BE00FE
:101430003B08BD00BB01BC01831202308316D800FB
:101440008A118312A9218A158A11C5218A1583164A
:10145000D001CF01CE0183122B088316CD00D2011B
:1014600083122A08831652078312CF0083164D0871
:101470008312D000003003180130D00783164E08C5
:101480008312D100003003180130D10783164F08B2
:101490008312D200003003180130D2077408203CB8
:1014A000031D702A83163B088312CF0783163C085E
:1014B00003183C0F5C2A5F2A8312D00783163D086D
:1014C00003183D0F642A672A8312D10783163E084A
:1014D00003183E0F6C2A6F2A8312D20783168312D9
:1014E0008316D001CF01CE0183122A088316CD00C6
:1014F000D401D301D20183122B088316D1005308E3
:10150000FA005208F9005108F800F70177084D0772
:10151000D6004E08D70051080318510FD7074F08BF
:10152000D80052080318520FD8075008D9005308A2
:101530000318530FD9075908DD005808DC00570875
:10154000DB005608DA00E101E001DF0183122C081C
:101550008316DE008A11831266228A157A088316A2
:10156000DA007908D9007808D8007708D700831204
:101570002D0883165707DB005808DC0083122E085D
:1015800003182E0FC42AC72A8316DC07831283167A
:101590005908DD00003003180130DD075A08DE006D
:1015A000003003180130DE078312310883165B0711
:1015B0008312BB0083165C088312BC003208031838
:1015C000320FBC0783165D088312BD00003003187C
:1015D0000130BD0783165E088312BE000030031879
:1015E0000130BE078A11C5218A153F3084002A08C0
:1015F0008000403084002B0880008A11C5218A15A4
:10160000413084002A088000423084002B0880008A
:101610008A11DC218A150130F8008316162B8312FB
:101620008A11DC218A150030F800831683120034F9
:10163000941603108316C80DC90DCA0DCB0D831265
:10164000051013085130930083161418292B8312A8
:10165000242BCA3084000008D0008312130883169C
:1016600050088312930083161418382B8312332BDF
:10167000C93084000008D000831213088316500874
:101680008312930083161418472B8312422BC83001
:1016900084000008D00083121308831650088312B8
:1016A000930083161418562B8312512B83121308A0
:1016B0009301831614185E2B8312592B831213087F
:1016C000FF30930083161418672B8312622BDC0102
:1016D0008A11831244208A15780B712B0130F8008F
:1016E000D52BFE308316DC008A11831244208A1524
:1016F000780B7D2B0130F800D52B941285118316C1
:10170000CD011030CC00CC08031D892BCD08031966
:10171000B42B8312051A8F2B8316892B8312831601
:10172000CF01CE01CF08031DAF2B4E081F3C031C79
:10173000AF2B83120616061206160612061606129E
:1017400006160612061606120616061206160612C9
:10175000061606128316CE0A0319CF0A922B4C08DE
:101760000319CD03CC03832B83128515941613081C
:10177000FF30930083161418BF2B8312BA2B8312E9
:101780001308FF30930083161418C82B8312C32B41
:10179000831205141308FF30930083161418D22BFC
:1017A0008312CD2B0030F800831200348316C7015A
:1017B000C5010230C800C9010830CA000430CB009E
:1017C0008A118312D0258A1501308316C8008A1128
:1017D00083127E258A1502308316C8000B30C9009B
:1017E000831229088316CA00831229088316CB00A6
:1017F0008A118312D0258A1501308316C8008A11F8
:1018000083127E258A1583163B08CB003A08CA004E
:101810003908C9003808C800CF01CE01CD018312B4
:101820002C088316CC008A11831222228A157A088A
:101830008316BB007908BA007808B9007708B800A9
:101840003F08CB003E08CA003D08C9003C08C8005C
:10185000CF01CE01CD0183122C088316CC008A1152
:10186000831222228A157A088316BF007908BE00E7
:101870007808BD007708BC003B083F02031C7A2DA6
:10188000031D522C3A083E02031C7A2D031D522CD4
:1018900039083D02031C7A2D031D522C38083C02E6
:1018A000031C7A2DC70183122C08831647020318E4
:1018B000152D023083124F028316C0008312500888
:1018C0008316C1000030031C0130C102831251088D
:1018D0008316C2000030031C0130C202831252087A
:1018E0008316C3000030031C0130C30283122C088E
:1018F000F700F801F901FA017A088316CB0079089C
:10190000CA007808C9007708C8004308DD0042080B
:10191000DC004108DB004008DA004B08E1004A081F
:10192000E0004908DF004808DE008A1183126622C1
:101930008A157A088316C3007908C2007808C100A6
:101940007708C00083124B088316C00783124C0827
:1019500003184C0FAC2CAF2C8316C10783124D0813
:1019600003184D0FB42CB72C8316C20783124E08F0
:1019700003184E0FBC2CBF2C8316C307831283168B
:10198000F801F901FA014708C00778080318780F31
:10199000C10779080318790FC2077A0803187A0F6C
:1019A000C3074308CB004208CA004108C9004008E9
:1019B000C8008312182378088316C500450BED2C48
:1019C0004308CB004208CA004108C9004008C800CB
:1019D0008312182378088316C500450BFB2C0230B0
:1019E000C8000B30C900FE30CA00CB008A11831238
:1019F000D0258A1583168312061B012D6E30F80040
:101A00007D2D861B122DC308031D0F2DC408031D39
:101A10000F2DC508031D0F2DC6080319122D703098
:101A2000F8007D2D8316C70A532C83125208D60066
:101A30005108D5005008D4004F08D300560883162B
:101A4000D000831255088316CF00831254088316E2
:101A5000CE00831253088316CD008A1183125926B3
:101A60008A157A08D2007908D1007808D000770862
:101A7000CF0002308316C8000B30C900831229083A
:101A80008316CA00831229088316CB008A11831299
:101A9000D0258A150618702D14308316C8008A11B7
:101AA00083127E258A1506185D2D14308316C80012
:101AB0008A1183127E258A15532D061C672D14303A
:101AC0008316C8008A1183127E258A155D2D061C97
:101AD000672D14308316C8008A1183127E258A155B
:101AE00001308316B8070318B90A0319BA0A031993
:101AF000BB0A3C2C7330F8008312003484011F3081
:101B0000830583161F08C0399F009B01073083128D
:101B10009F008517FF30FC00703083168500EB3086
:101B200086000730810072308F00C03083128B0432
:101B30008B16851485152330A9008A1171288A1502
:101B400078088316B100310BA62DA52D8A118312BA
:101B5000922A8A158A11052E8A15C601C501C4016B
:101B60000130C3008A11ED2E8A157208DA0071085F
:101B7000D9007008D8006F08D70073308316B00002
:101B8000B1018312061B402E8316B20132080F3CAE
:101B9000031CD02DA030320784008001B20AC62D6C
:101BA0008312061BD82DF60AF50A8316D02D831250
:101BB000061F3F2E861F3F2E8A117F2F8A157A0817
:101BC000C6007908C5007808C4007708C300460835
:101BD0008316B700831245088316B60083124408A3
:101BE0008316B500831243088316B4008312412084
:101BF00078088316B100310B3E2E0310FA018312D0
:101C0000420CF900410CF800400CF7003B0783162A
:101C1000B40083123C088316B50078080318780FC7
:101C2000B50783123D088316B60079080318790FAB
:101C3000B60783123E088316B7007A0803187A0F96
:101C4000B70783123E088316BB0083123D08831634
:101C5000BA0083123C088316B90083123B0883162E
:101C6000B8003708BF003608BE003508BD0034088C
:101C7000BC008312D62378088316B0008312D82DB7
:101C8000061B8E2E78308316B200B2080319562E2A
:101C90000330C8008A1183127E258A15061F532E31
:101CA0008316562E83128316B203452E8312061B0B
:101CB0008E2E01308316C8008A1183127E258A1564
:101CC0008316B20A32080F3C031D8C2EB20101307C
:101CD0008312C3070318C40A0319C50A0319C60AE5
:101CE00062084602031C8B2E031D862E61084502E6
:101CF000031C8B2E031D862E60084402031C8B2EB2
:101D0000031D862E43085F0203188B2EC601C501F2
:101D1000C4010130C3008316562E8312861BD52EB4
:101D200078308316B200B2080319A42E0330C8001D
:101D30008A1183127E258A15861FA12E8316A42E52
:101D400083128316B203932E8312861BD52E013085
:101D50008316C8008A1183127E258A158316B20A5B
:101D600032080F3C031DD32EB201FF308312C3078C
:101D7000031CC407031CC507031CC607C308031DB7
:101D8000D22EC408031DD22EC508031DD22EC608AC
:101D9000031DD22E6208C6006108C5006008C40099
:101DA0005F08C3008316A42E8312061F772F861F99
:101DB000772F8316B201831246088316B700831269
:101DC00045088316B600831244088316B5008312B3
:101DD00043088316B4008312412078088316B100AB
:101DE0003108023C031DFE2E8312C601C501C40149
:101DF0000130C30073308316B000412F310B412FE7
:101E00000310FA018312420CF900410CF800400C57
:101E1000F7003B078316B40083123C088316B50015
:101E200078080318780FB50783123D088316B600AB
:101E300079080318790FB60783123E088316B70096
:101E40007A0803187A0FB70783123E088316BB007F
:101E500083123D088316BA0083123C088316B9002A
:101E600083123B088316B8003708BF003608BE004F
:101E70003508BD003408BC008312D62378088316C9
:101E8000B00030086E3C0319492F3008733C031D25
:101E9000542F01308312C3070318C40A0319C50A5B
:101EA0000319C60A772F83163008703C031D782F5C
:101EB0008312C608031D662FC508031D662FC408BC
:101EC000031D662F4308013C03186F2FFF30C30723
:101ED000031CC407031CC507031CC607772F620831
:101EE000C6006108C5006008C4005F08C30083160F
:061EF0008312402E630086
:10420000D0004B0089006E00DA00F700A50017000F
:10421000F800D800CC003B0076002300C1001D0050
:1042200053009E005D003900E000C2000300CF0093
:10423000CD009500CB0016008100AB000A008E0077
:10424000FB006300F900F400900010001100EE0084
:104250002500C5006F0097000400C000680007003B
:104260005F0096004300650045000F008400BA001F
:1042700057009C00CE001B00A6001400B600A3004F
:104280005C00C6007700D500B4003D009800270010
:10429000B90013003A002D00210040001800A000D2
:1042A0002800DE00AC008300E300DD0069006C0044
:1042B000B100B70049002B009D000C00C700710041
:1042C0000900F5007E0082006A007800D200D70065
:1042D0001F00A700F6004C008B00C300EF00320067
:1042E000E500A90037007A00D4001E007000060027
:1042F00055008D005200EC00150020005900DB0035
:10430000AD00BC007F004A00D600BB00BE00B0007C
:104310003E007B00BD007900B8009400E10022005F
:104320000100C4001C0031002E004F004D0036007B
:104330007500F000AF00F2008C00E7000D00800077
:10434000190061009200E400B300740046003500DB
:10435000B2001200FE004E006D009B00F100E9006B
:104360005100FF009F00CA0066000200AE000E0070
:104370009300EA003C00080054003400620064002E
:10438000E6009100D3007D000B00B500A4001A00E8
:104390005A008600A10024004700DF008F00E800DB
:1043A00088003F00440033006000F30042004100F9
:1043B000EB002F009A00ED00FC004800D1007200D5
:1043C0008A0073005600FA0005005E0085002A008E
:1043D0002C005800E2006700FD007C00A8005B0094
:1043E0003000D900380050008700DC006B00BF00AF
:1043F000C900A20099002600AA002900C8000000F8
:02400E00383F39
:00000001FF
